:1000000000308A0047280000FF00030E8301A10092
:100010007F08A0000A08A8008A01A00E0408A20018
:100020007708A3007808A4007908A5007A08A6003C
:100030007B08A700831383128C308400801C222845
:100040008C183528220884002308F7002408F800BB
:100050002508F9002608FA002708FB0028088A006E
:10006000210E8300FF0E7F0E09000130A90703183F
:10007000AA0A0319AB0A0319AC0A85141030F70059
:10008000F70B4028000085108C108A11222884016B
:100090001F30830507309F00F93083168500FF303D
:1000A0008600073083129F008030831681000E3057
:1000B00083129200F93083169200C03083128B04B1
:1000C0000511AC01AB01AA01A90183168C1483129E
:1000D000AC08031D7B28AB08031D7B282A08743C51
:1000E000031C7B28031D78282908033C031C7B285C
:0C00F00083166728831205156300630067
:00000001FF
